:0200000480007A
:100000006F008004732F2034930F80006308FF0378
:10001000930F90006304FF03930FB0006300FF038E
:10002000130F000063040F0067000F00732F2034CC
:1000300063540F006F00400093E19153171F0000BD
:1000400023223FFC6FF09FFF93000000130100008C
:10005000930100001302000093020000130300004C
:100060009303000013040000930400001305000034
:10007000930500001306000093060000130700001C
:100080009307000013080000930800001309000004
:1000900093090000130A0000930A0000130B0000EC
:1000A000930B0000130C0000930C0000130D0000D4
:1000B000930D0000130E0000930E0000130F0000BC
:1000C000930F0000732540F16310050097020000B4
:1000D000938202017390523073500018970200000F
:1000E00093824202739052309B021000939252030B
:1000F0009382F2FF7390023B9302F0017390023AF5
:100100007350403097020000938242017390523046
:10011000735020307350303093010000970200007C
:10012000938282EE73905230130510001315F5017F
:10013000635C05000F00F00F930110009308D005D9
:10014000130500007300000093020000638A0200A0
:1001500073905210B7B200009B82921073902230BD
:100160007350003097020000938242017390123462
:10017000732540F1730020309301200093000000AC
:100180001301100063E62000631C30366316300054
:10019000E3EE20FE63163036930130009B00100022
:1001A000939000029380E0FF1B01100013110102E5
:1001B0001301F1FF63E6200063143034631630004E
:1001C000E3EE20FE631E30329301400093000000F6
:1001D0001B011000131101021301F1FF63E620005F
:1001E0006310303263163000E3EE20FE631A3030C5
:1001F00093015000930010001301000063E42000FD
:1002000063143000631E302EE3EE20FE9301600085
:100210009B001000939000029380F0FF1B011000E0
:10022000131101021301E1FF63E4200063143000A5
:100230006318302CE3EE20FE930170009B00100049
:10024000939000029380F0FF1301000063E420000C
:10025000631430006316302AE3EE20FE9301800021
:100260009B0010009390F001370100801B01F1FF0B
:1002700063E420006314300063143028E3EE20FEB2
:1002800093019000130200009B00F0009390C001C6
:100290001B01F0001311C1011301F1FF63E22026DD
:1002A0001302120093022000E31052FE9301A000FB
:1002B000130200009B00F0009390C0011B01F000AE
:1002C0001311C1011301F1FF1300000063EA2022A2
:1002D0001302120093022000E31E52FC9301B000AF
:1002E000130200009B00F0009390C0011B01F0007E
:1002F0001311C1011301F1FF1300000013000000EE
:1003000063E020201302120093022000E31C52FC41
:100310009301C000130200009B00F0009390C00105
:10032000130000001B01F0001311C1011301F1FFC4
:1003300063E8201C1302120093022000E31E52FC0B
:100340009301D000130200009B00F0009390C001C5
:10035000130000001B01F0001311C1011301F1FF94
:100360001300000063EE2018130212009302200015
:10037000E31C52FC9301E000130200009B00F0001C
:100380009390C00113000000130000001B01F00057
:100390001311C1011301F1FF63E4201613021200CF
:1003A00093022000E31C52FC9301F00013020000B2
:1003B0009B00F0009390C0011B01F0001311C101DC
:1003C0001301F1FF63EE20121302120093022000CA
:1003D000E31052FE93010001130200009B00F000A5
:1003E0009390C0011B01F0001311C1011301F1FF33
:1003F0001300000063E62010130212009302200095
:10040000E31E52FC93011001130200009B00F00058
:100410009390C0011B01F0001311C1011301F1FF02
:10042000130000001300000063EC200C1302120004
:1004300093022000E31C52FC9301200113020000F0
:100440009B00F0009390C001130000001B01F0001E
:100450001311C1011301F1FF63E4200A130212001A
:1004600093022000E31E52FC9301300113020000AE
:100470009B00F0009390C001130000001B01F000EE
:100480001311C1011301F1FF1300000063EA2006FC
:100490001302120093022000E31C52FC930140015E
:1004A000130200009B00F0009390C00113000000B5
:1004B000130000001B01F0001311C1011301F1FF33
:1004C00063E020041302120093022000E31C52FC9C
:1004D00093001000636A1000938010009380100056
:1004E0009380100093801000938010009380100080
:1004F0009303300093015001639470006310300245
:100500000F00F00F638001009391110093E111003F
:100510009308D00513850100730000000F00F00F51
:10052000930110009308D00513050000730000002C
:0C053000731000C000000000000000007C
:1010000000000000000000000000000000000000E0
:1010100000000000000000000000000000000000D0
:1010200000000000000000000000000000000000C0
:1010300000000000000000000000000000000000B0
:081040000000000000000000A8
:040000058000000077
:00000001FF
